:1000000008308A00952D0000FF00030E8301A10037
:100010000A08A0008A010408A2007708A300780853
:10002000A4007908A5007A08A6007B08A70083131E
:1000300083128B1E1D280B193028220884002308E8
:10004000F7002408F8002508F9002608FA00270818
:10005000FB0020088A00210E8300FF0E7F0E09009E
:100060008A110A1279290A108A100A113A3E0318D5
:100070008A0A8200D0344B3489346E34DA34F7344F
:10008000A5341734F834D834CC343B3476342334A4
:10009000C1341D3453349E345D343934E034C234B9
:1000A0000334CF34CD349534CB3416348134AB346F
:1000B0000A348E34FB346334F934F434903410341D
:1000C0001134EE342534C5346F3497340434C034DD
:1000D000683407345F3496344334653445340F3420
:1000E0008434BA3457349C34CE341B34A63414349C
:1000F000B634A3345C34C6347734D534B4343D34A8
:1001000098342734B93413343A342D3421344034FC
:100110001834A0342834DE34AC348334E334DD3492
:1001200069346C34B134B73449342B349D340C34D5
:10013000C73471340934F5347E3482346A34783407
:10014000D234D7341F34A734F6344C348B34C33410
:10015000EF343234E534A93437347A34D4341E34AD
:100160007034063455348D345234EC341534203424
:100170005934DB34AD34BC347F344A34D634BB34E8
:10018000BE34B0343E347B34BD347934B834943426
:10019000E13422340134C4341C3431342E344F342D
:1001A0004D3436347534F034AF34F2348C34E734B3
:1001B0000D348034193461349234E434B3347434FB
:1001C00046343534B2341234FE344E346D349B34FC
:1001D000F134E9345134FF349F34CA346634023484
:1001E000AE340E349334EA343C340834543434346A
:1001F00062346434E6349134D3347D340B34B53412
:10020000A4341A345A348634A13424344734DF34C5
:100210008F34E83488343F34443433346034F33436
:1002200042344134EB342F349A34ED34FC344834C6
:10023000D13472348A3473345634FA3405345E342B
:1002400085342A342C345834E2346734FD347C3419
:10025000A8345B343034D934383450348734DC3407
:100260006B34BF34C934A23499342634AA342934C7
:10027000C8340034071183166708831293000330D3
:10028000F700F70B4129000000008316680883126D
:1002900093000330F700F70B4B2900000000831692
:1002A0006908831293000330F700F70B552900000B
:1002B0000000EC3084001308800083166A08831263
:1002C00093000330F700F70B632900000000EB30C8
:1002D0008400130880000730F700F70B6D29000039
:1002E0000000071583166B08F8006C08F9008312EC
:1002F0000034861A952903308316E7000B30E80096
:10030000E901EA0183123A217808F500750F89297D
:100310008A29F50A02308316E7000B30E8007508D9
:10032000E9007508EA0083123A21061AB129033060
:100330008316E7000B30E800E901EA0183123A2155
:100340007808F500F5080319A629F503023083168D
:10035000E7000B30E8007508E9007508EA00831231
:100360003A210B118A110A121D28F93083168600D2
:10037000831206110330F700F70BBC290615003471
:10038000F93083168600D23087002230850088013C
:10039000890106309F00810083129F0107151830E4
:1003A00085008901B521981783169901181618132D
:1003B00098179816141783129416A8018B1BA81768
:1003C0008B1302308316E7000B30E8002030E90081
:1003D000EA0083123A21A81B8B178A150A129F2D57
:1003E000C930840000080319042A0130F800F7011D
:1003F000F70BF829F80BF7294A30F700F70BFE291D
:1004000000000000800BF5290034851E052A003409
:100410000522FF30831688008312880185110808A1
:10042000AA008515052285110808AB0085158316DD
:1004300088018312003485150516861089018518F8
:100440001F2A05150630F700F70B242A00000511B6
:1004500064308316C9008312F02107308900EC3024
:10046000880005220512051608228A150A12A72DF2
:100470000F308316DB05E030DB04DB30840000083E
:10048000831288000630890005120516DA308400D0
:10049000000888000530890005120516D93084004F
:1004A000000888000430890005120516D830840041
:1004B0000008880003308900051205160130880005
:1004C00002308900051205162030880007308900A7
:1004D00005120516890100348316D8080319802AED
:1004E0008312851A752A8316702A85118515851E33
:1004F000772A851185158316D80383126C2A8316F3
:1005000083120034F701F801F901FA018316D101D1
:10051000D201D301D40150084F044E044D040319F5
:10052000C12A2030D5000310C90DCA0DCB0DCC0D4A
:10053000D10DD20DD30DD40D50085402031DAA2A9B
:100540004F085302031DAA2A4E085202031DAA2A6D
:100550004D085102031CBB2A4D08D1024E08031C52
:100560004E0FD2024F08031C4F0FD3025008031C3A
:10057000500FD4020314F70DF80DF90DFA0DD50B39
:10058000932A0000D1308400831200342030831677
:10059000E600E201E301E401E5015D08FA005C0820
:1005A000F9005B08F8005A08F7000310771CE62AE8
:1005B0005E08E2075F0803185F0FE307600803188F
:1005C000600FE40761080318610FE507E50CE40C10
:1005D000E30CE20CFA0CF90CF80CF70CE60BD52A3C
:1005E00083120034AE01AD018316DB01DA01D901BB
:1005F000D80183123822E3308316D80083126C228C
:1006000008228316B90183122B088316B8008312BF
:10061000AE00AD012A08AD070318AE0A8316BB0170
:10062000BA0183122E088316B90083122D0883168F
:10063000B8003B08DB003A08DA003908D90038086E
:10064000D8008312382205308316D80083126C221A
:100650000822C6012B08C50008228316B90183129F
:100660002A088316B800FA0000308312C507031861
:10067000C60A7A08C6072B08AC0008228316B901FF
:1006800083122B088316B800BB00BA0183122A0814
:1006900083163A078312B30083163B088312B40013
:1006A0000318B40A08222A08F300E601E501E40170
:1006B0002B08E30008228316B90183122A08831647
:1006C000B800FA0000308312E3077A0803187A0FA3
:1006D000E407003003180130E5070030031801304B
:1006E000E607082208228316B90183122B08831615
:1006F000B800FA00003083122A07E7007A08E80001
:10070000003003180130E807E901EA0106308316DA
:10071000D80083126C220822EE01ED01EC01EB01FE
:100720008316BB01BA01B90183122B088316B800E6
:100730003A08FA003908F9003808F800F701770894
:1007400083122A07EB007808EC0000300318013010
:10075000EC077908ED00003003180130ED077A0846
:10076000EE00003003180130EE076E088316B70064
:1007700083126D088316B60083126C088316B500C9
:1007800083126B088316B400831208228316BB0100
:10079000BA01B90183122B088316B8003A08FA008F
:1007A0003908F9003808F800F701770883122A079A
:1007B000EB007808EC00003003180130EC077908F2
:1007C000ED00003003180130ED077A08EE0000302C
:1007D00003180130EE076C08EE006B08ED00EB012A
:1007E000EC01831634088312EB07831635080318CF
:1007F000350FFB2BFE2B8312EC07831636080318EC
:10080000360F032C062C8312ED07831637080318C6
:10081000370F0B2C0E2C8312EE078316831208223F
:10082000082208228316BB01BA01B90183122B08E2
:100830008316B8003A08FA003908F9003808F800B9
:10084000F701770883122A07EF007808F0000030DC
:1008500003180130F0077908F10000300318013067
:10086000F1077A08F200003003180130F20772082D
:100870008316B7007108B6007008B50083126F08C0
:100880008316B400831208228316BB01BA01B90192
:1008900083122B088316B8003A08FA003908F900C9
:1008A0003808F800F701770883122A07EF00780864
:1008B000F000003003180130F0077908F100003033
:1008C00003180130F1077A08F200003003180130F4
:1008D000F2077008F2006F08F100EF01F0018316D3
:1008E00034088312EF07831635080318350FF00715
:1008F00036080318360FF10737080318370FF207C9
:1009000072088312DA007108D9007008D8006F08E5
:10091000D70033082D07C7002E08C8003408031875
:10092000340FC807C901CA01630D8316B8008312CA
:10093000640D8316B9008312650D8316BA00831205
:10094000660D8316BB00B80DB90DBA0DBB0DB80D01
:10095000B90DBA0DBB0DB80DB90DBA0DBB0DB80D63
:10096000B90DBA0DBB0DE030B80501308312450258
:10097000F7004608FA000030031C0130FA0277083D
:1009800083163807BC003908BD007A0803187A0FAF
:10099000BD073A08BE00003003180130BE073B080F
:1009A000BF00003003180130BF073F08CC003E08ED
:1009B000CB003D08CA003C08C900D001CF0183121A
:1009C00046088316CE00831245088316CD00831295
:1009D00082227808B0007708AF00E708031DF92CE1
:1009E000E808031DF92CE908031DF92CEA0803198E
:1009F0003A2D1030F4008316DD01DC01DB017308B1
:100A0000DA0083126A088316E100831269088316EC
:100A1000E000831268088316DF00831267088316DC
:100A2000DE008312C622770833078316B8008312CC
:100A300034088316B90078080318780FB9077908C5
:100A4000BA00003003180130BA077A08BB00003042
:100A500003180130BB0783122F088316380783124F
:100A6000B100831639088312B2000318B20A3008A5
:100A7000B2077A2D2030F4008316DD01DC01DB01A2
:100A80007308DA0083126E088316E10083126D0882
:100A90008316E00083126C088316DF0083126B0854
:100AA0008316DE008312C622770833078316B80048
:100AB000831234088316B90078080318780FB90731
:100AC0007908BA00003003180130BA077A08BB0071
:100AD000003003180130BB0783122F088316380734
:100AE0008312B100831639088312B2000318B20AC8
:100AF0003008B2078316BB01BA01B9017308B80008
:100B00003B08DD003A08DC003908DB003808DA0071
:100B100083126A088316E100831269088316E000D5
:100B2000831268088316DF00831267088316DE00CD
:100B30008312C62277083307B5003408B600780858
:100B40000318780FB6077908B70000300318013092
:100B5000B7077A08B800003003180130B8078316C9
:100B6000BB01BA0183122E088316B90083122D0827
:100B70008316B8008312F901FA0131088316380789
:100B80008312CB00831639088312CC003208031875
:100B9000320FCC0783163A088312CD007908031868
:100BA000790FCD0783163B088312CE007A0803180D
:100BB0007A0FCE070034871CF82D8316CA01C901AD
:100BC0004A08073C031CF72DCB0183120714831638
:100BD0004B0883129900000000000710000000007D
:100BE000000000008316C90A0319CA0AE02D831207
:100BF0000034A8018B1BA8178B1302308316E70063
:100C0000E8010330E9000430EA0083123A21A81B0E
:100C10008B17A8018B1BA8178B1302308316E700D4
:100C2000E8010330E900EA0183123A21A81B8B177F
:100C3000DB2500348316D201D1017408203C031D4A
:100C4000262E0310CD0DCE0DCF0DD00DCD3084004E
:100C50000008D7004E08CD004F08CE005008CF0046
:100C6000D001831247088316CD0783124808031862
:100C7000480F3B2E3E2E8316CE07831249080318D9
:100C8000490F432E462E8316CF0783124A080318B6
:100C90004A0F4B2E4E2E8316D00783128316500810
:100CA000DB004F08DA004E08D9004D08D800831247
:100CB000382283165708D80083126C220822831624
:100CC000D90183122B088316D800DB00DA01FA0160
:100CD00083122A0883165A07D1005B08D200031832
:100CE000D20A7A08D2077408103C031D7E2E5108E0
:100CF000F7005208F800F901FA01B82E8312082211
:100D00008316D601D501D401D301D90183122B0852
:100D10008316D800DB00DA01FA0183122A08831651
:100D20005A07D3005B08D4007A0803187A0FD40757
:100D3000D501D6015408D6005308D500D301D401FB
:100D4000F901FA015108D30752080318520FD407CA
:100D500079080318790FD5077A0803187A0FD60790
:100D60005308F7005408F8005508F9005608FA002F
:100D7000831200347208DA007108D9007008D800B4
:100D80006F08D7008316B701B601B501B40183120D
:100D90005A08DE005908DD005808DC005708DB005F
:100DA0005E088316D00083125D088316CF0083127D
:100DB0005C088316CE0083125B088316CD00831275
:100DC0001A267A08DA007908D9007808D800770856
:100DD000D70057088316B800831258088316B90045
:100DE000831259088316BA0083125A080F398316E2
:100DF000BB000130B4070318B50A0319B60A03197A
:100E0000B70A3B080F3C031C172F031DC72E3A08D7
:100E1000FF3C031C172F031DC72E3908FF3C031C82
:100E2000172F031DC72E3808EE3C0318C72E3708AE
:100E3000DD003608DC003508DB003408DA00E101AB
:100E4000E001DF0183122C088316DE008312C62224
:100E50007A08E2007908E1007808E0007708DF000E
:100E6000DF0DE00DE10DE20DDF0DE00DE10DE20D16
:100E7000DF0DE00DE10DE20DDF0DE00DE10DE20D06
:100E8000F030DF05FF30DF07031CE007031CE1073C
:100E9000031CE2078A150A12D42DFF308316B7000F
:100EA000B6008312E208031DB12FE108031DB12F24
:100EB00060088316370203185F2F8312B12F031DBA
:100EC000672F360883125F020318B12F8316BA0109
:100ED0008312A91F6F2F01308316BA008312A91E37
:100EE000752F01308316BA068312291E7B2F01301D
:100EF0008316BA068312291D812F01308316BA0684
:100F000083120310A90D83163A088312A904290835
:100F1000F80078088316B800B80E0F30B805A03076
:100F200038078400000F952FAF2FA03038078400BA
:100F30000008800AB9007608B907390883123320FF
:100F4000F8008316B7017808B600BB013808B50071
:100F5000B4013408B6070318B70A3508B707512F8C
:100F6000831283163608F7003708F800F901FA01F2
:100F700083128A150A12022EF801F901F701FA010B
:100F800083165008031DC72F4F080319E12F103097
:100F9000D1000310CD0DCE0DF70DFA0D50087A02D9
:100FA000031DD42F4F087702031CDD2F4F08F702D3
:100FB000031CFA035008FA020314F80DF90DD10BC3
:100FC000C92F000083128A150A1299281030F700E1
:100FD000FA018316D101CE0CCD0C031CF52F4F085E
:100FE000FA070318D10A5008D107D10CFA0CF90CF2
:0E0FF000F80CF70BEB2F83128A150A12AB28B0
:101000008316C601C501C401C3017408103C031D49
:101010006728370CFA00360CF900350CF800340C50
:10102000F700FA0CF90CF80CF70CFA0CF90CF80CA8
:10103000F70CFA0CF90CF80CF70C0F30FA057708DE
:10104000831235078316CD00831236088316CE002F
:1010500078080318780FCE07831237088316CF005D
:1010600079080318790FCF07831238088316D00048
:101070007A0803187A0FD00783122D0883164D07BC
:10108000D1004E08D20083122E0803182E0F4928D3
:101090004C288316D207831283164F08D3000030E2
:1010A00003180130D3075008D40000300318013072
:1010B000D4075408DB005308DA005208D90051085D
:1010C000D8008A11831238228A159A298316720849
:1010D0008312DA007108D9007008D8006F08D700B1
:1010E0008316370CFA00360CF900350CF800340C76
:1010F000F700FA0CF90CF80CF70CFA0CF90CF80CD8
:10110000F70CFA0CF90CF80CF70C7708C900780802
:10111000CA004A08CC004908CB004A08CE0049085A
:10112000CD00D00183122C088316CF008A118312C0
:10113000BC2F8A1579088316CA007808C9004A08A6
:10114000CE004908CD00D00183122C088316CF00B1
:101150008A118312E62F8A1579088316C800780849
:10116000C70047084B02C7004808031C480FBA28AD
:101170004C08BB284C02C800C908031DC228CA0875
:101180000319FB2883125A08DE005908DD005808AD
:10119000DC005708DB005E088316D00083125D0870
:1011A0008316CF0083125C088316CE0083125B087F
:1011B0008316CD008A1183121A268A157A08DA005E
:1011C0007908D9007808D8007708D700570883161F
:1011D000C300831258088316C4008312590883166B
:1011E000C50083125A080F398316C600490803192F
:1011F000CA03C903BC2846080E3C03181729FF3A46
:10120000031D14294508FE3C03181729FF3A031D46
:1012100014294408FE3C03181729FF3A031D14291A
:101220004308EF3C031817290230F800222B023044
:10123000831257028316BF00831258088316C0001A
:101240000030031C0130C002831259088316C1000C
:101250000030031C0130C10283125A088316C200F9
:101260000030031C0130C20283122C08F700F80181
:10127000F901FA017A088316D0007908CF007808BE
:10128000CE007708CD004208DD004108DC004008B0
:10129000DB003F08DA005008E1004F08E0004E088C
:1012A000DF004D08DE008A118312C6228A157A08F3
:1012B0008316C2007908C1007808C0007708BF0013
:1012C00083124B088316BF0783124C0803184C0F78
:1012D0006A296D298316C00783124D0803184D0F24
:1012E000722975298316C10783124E0803184E0F01
:1012F0007A297D298316C20783128316F901FA0120
:101300004708BF0748080318480FC00779080318A3
:10131000790FC1077A0803187A0FC2074208DB0069
:101320004108DA004008D9003F08D8008A1183122A
:1013300038228A15831634080F39CD003508003954
:10134000CE0036080039CF0037080039D0004D0DE7
:10135000D1004E0DD2004F0DD300500DD400D10D51
:10136000D20DD30DD40DD10DD20DD30DD40DD10D81
:10137000D20DD30DD40DF030D1055108D8008A110B
:1013800083126C228A158A1108228A15AA08031D65
:10139000CE290030F8008316222B83122A08E53C60
:1013A00003191F2B8A1108228A158A1108228A150F
:1013B0008A1108228A158A1108228A152A0883169A
:1013C000B80083122B088316B9008A1183120822F1
:1013D0008A152A088316BA0038086D3C0319F429C7
:1013E00038084D3C031D1E2B3908503C0319FC29BD
:1013F0003908703C031D1E2B3A08333C031D1E2B7D
:101400000430D8008A1183126C228A158A110822AE
:101410008A157408203C031D292A8316CE018312E5
:101420002B088316CD00D000CF0183122A08831623
:101430004F07BB005008BC00003003180130BC0748
:10144000BD01BE013C08BE003B08BD00BB01BC01A4
:10145000831202308316D8008A1183126C228A15F7
:101460008A1108228A158316D001CF01CE0183127A
:101470002B088316CD004F08D5004E08D4004D0828
:10148000D300D20183122A08831652078312CF0099
:10149000831653088312D000003003180130D007A0
:1014A000831654088312D100003003180130D1078D
:1014B000831655088312D200003003180130D2077A
:1014C0007408203C031D822A83163B088312CF0731
:1014D00083163C0803183C0F6E2A712A8312D0072A
:1014E00083163D0803183D0F762A792A8312D10707
:1014F00083163E0803183E0F7E2A812A8312D207E4
:10150000831683128316D001CF01CE0183122A08DD
:101510008316CD00D401D301D20183122B08831688
:10152000D1005308FA005208F9005108F800F701F9
:1015300077084D07D6004E08D70051080318510F01
:10154000D7074F08D80052080318520FD807500881
:10155000D90053080318530FD9075908DD0058085C
:10156000DC005708DB005608DA00E101E001DF018A
:1015700083122C088316DE008A118312C6228A1574
:101580007A088316DA007908D9007808D800770835
:10159000D70083122D0883165707DB005808DC009C
:1015A00083122E0803182E0FD62AD92A8316DC0799
:1015B000831283165908DD00003003180130DD075F
:1015C0005A08DE00003003180130DE0783123108AC
:1015D00083165B078312B90083165C088312BA0076
:1015E00032080318320FBA0783165D088312BB0056
:1015F000003003180130BB0783165E088312BC005D
:10160000003003180130BC078A1108228A153D30CA
:1016100084002A0880003E3084002B0880008A1154
:1016200008228A153F3084002A0880004030840058
:101630002B0880000130F8008316222B8312003023
:10164000F8008316831200348316C801C5010130E7
:10165000C6008A118312F9258A1583163B08CC002F
:101660003A08CB003908CA003808C900D001CF01B8
:10167000CE0183122C088316CD008A118312822298
:101680008A157A088316BB007908BA007808B90071
:101690007708B8003F08CC003E08CB003D08CA00E0
:1016A0003C08C900D001CF01CE0183122C0883165B
:1016B000CD008A11831282228A157A088316BF0010
:1016C0007908BE007808BD007708BC003B083F02DF
:1016D000031C6F2D031D7C2B3A083E02031C6F2D4B
:1016E000031D7C2B39083D02031C6F2D031D7C2B31
:1016F00038083C02031C6F2DC80183122C08831686
:1017000048020318B52C023083124F028316C00022
:10171000831250088316C1000030031C0130C1023F
:10172000831251088316C2000030031C0130C2022C
:10173000831252088316C3000030031C0130C30219
:1017400083122C08F700F801F901FA017A088316D0
:10175000CC007908CB007808CA007708C900430894
:10176000DD004208DC004108DB004008DA004C08DC
:10177000E1004B08E0004A08DF004908DE008A115A
:101780008312C6228A157A088316C3007908C2001C
:101790007808C1007708C00083124B088316C00781
:1017A00083124C0803184C0FD62BD92B8316C10774
:1017B00083124D0803184D0FDE2BE12B8316C20751
:1017C00083124E0803184E0FE62BE92B8316C3072E
:1017D00083128316F801F901FA014808C007780856
:1017E0000318780FC10779080318790FC2077A0820
:1017F00003187A0FC307460B192C4308CC00420884
:10180000CB004108CA004008C9002030CD00CD08F7
:101810000319182C0830CE00CE080319162C8A1193
:10182000831208228A158316CE030C2CCD03072CB5
:10183000C6014308DB004208DA004108D90040082D
:10184000D8008A11831238228A1583164B14FF3070
:1018500088001030CA00CA080319572C8312871851
:10186000352C83164B102E2C831210308316C90092
:10187000C9080319552C8A11831205228A1585116E
:1018800007140808990085150710000000000000E3
:10189000000000008511071408089900851507103D
:1018A000000000008316C903382CCA032B2C8801C2
:1018B00000304B180130F800F8080319942CC50AC1
:1018C0004508783C0318932C8312A8018B1BA8179A
:1018D0008B1303308316E7000B30E800E901EA01BF
:1018E0008A1183123A218A15A81B8B177808F500F4
:1018F0008A11B5218A158A11F9258A15A8018B1B31
:10190000A8178B1302308316E7000B30E800750828
:10191000E9007508EA008A1183123A218A15A81B8A
:101920008B178316C5019B2CC5034508013C031C7E
:101930009B2C0230C5008312861BA12C6E30F80050
:10194000722D061BB22CC108031DAF2CC208031D4B
:10195000AF2CC308031DAF2CC4080319B22C703080
:10196000F800722D8316C80A7D2B83125208D60008
:101970005108D5005008D4004F08D30056088316EC
:10198000D000831255088316CF00831254088316A3
:10199000CE00831253088316CD008A1183121A26B3
:1019A0008A157A08D2007908D1007808D000770823
:1019B000CF008619652D83164410FA30C7008312B4
:1019C000A8018B1BA8178B1303308316E7000B307D
:1019D000E8000330E9001430EA008A1183123A214A
:1019E0008A15A81B8B177808F5008619092D083071
:1019F0008316C9008A118312F0218A158316C7083D
:101A0000031D062D8312061183164414C703831287
:101A1000F52C08308B0063008B018316441C5E2D6F
:101A20008312061501308316C9008A118312F02132
:101A30008A15A8018B1BA8178B1302308316E700A9
:101A4000E8010330E9000430EA008A1183123A21E8
:101A50008A15A81B8B1701308316C9008A118312BF
:101A6000F0218A15A8018B1BA8178B13023083164F
:101A7000E700E8010330E900EA018A1183123A2104
:101A80008A15A81B8B1701308316C9008A1183128F
:101A9000F0218A15A8018B1BA8178B13023083161F
:101AA000E7000B30E8007508E9007508EA008A11C4
:101AB00083123A218A15A81B8B1783168A11831269
:101AC000DB258A15C0308B048B1601308316B807CE
:101AD0000318B90A0319BA0A0319BB0A662B733033
:101AE000F8008312003405100830F80000000000F0
:101AF0000000F8178C2DF8138316B40C831203180A
:101B00000514031C051078178C2D7813F80B7C2D09
:101B100000000000000005141C308400840B8E2D92
:101B2000F81B7B2D781B852D003484011F30830525
:101B3000063083169F00831205148A11C0298A1566
:101B4000051685158610C601C5018A111B2A8A153E
:101B50008A11F2228A15C508031DB22D4608023CDF
:101B60000319B52D8A11F2228A158A11F9258A15D1
:101B70003030F500A8018B1BA8178B130230831699
:101B8000E7000B30E8007508E9007508EA008A11E3
:101B900083123A218A15A81B8B17C401C301C20105
:101BA0000130C1008A11BA2E8A157208DA00710854
:101BB000D9007008D8006F08D70073308316B000C2
:101BC000B101B301C03083128B048B16861B642EC7
:101BD0008316B20132080F3C031CF42DA0303207EB
:101BE00084008001B20AEA2D8312861BFC2DA90A0B
:101BF000F60A8316F42D8312861F632E061F632EAA
:101C00008A114D2F8A157A08C4007908C300780814
:101C1000C2007708C10044088316B7008312430846
:101C20008316B600831242088316B500831241085A
:101C30008316B4008312002078088316B100310B9C
:101C4000622E0310FA018312400CF9003F0CF800D9
:101C50003E0CF70039078316B40083123A08831646
:101C6000B50078080318780FB50783123B08831670
:101C7000B60079080318790FB60783123C0883165B
:101C8000B7007A0803187A0FB70783123C08831647
:101C9000BB0083123B088316BA0083123A088316EE
:101CA000B900831239088316B8003708BF00360818
:101CB000BE003508BD003408BC0083122423780818
:101CC0008316B0008312FC2D861BBC2E7830831641
:101CD000B200B20803197A2E0330C9008A118312A8
:101CE000F0218A15861F772E83167A2E831283168B
:101CF000B203692E8312861BBC2E01308316C900E5
:101D00008A118312F0218A158316B20A32080F3C19
:101D1000031DBA2EB20101308312C1070318C20A93
:101D20000319C30A0319C40A62084402031CB42E2F
:101D3000031DAA2E61084302031CB42E031DAA2E04
:101D400060084202031CB42E031DAA2E41085F0244
:101D50000318B42EC401C301C2010130C1007330A5
:101D60008316B4008312732566308316B400831281
:101D7000732583167A2E8312061B0D2F7830831657
:101D8000B200B2080319D22E0330C9008A1183129F
:101D9000F0218A15061FCF2E8316D22E83128316AA
:101DA000B203C12E8312061B0D2F01308316C9000A
:101DB0008A118312F0218A158316B20A32080F3C69
:101DC000031D0B2FB201FF308312C107031CC20792
:101DD000031CC307031CC407C108031D052FC20849
:101DE000031D052FC308031D052FC408031D052F60
:101DF0006208C4006108C3006008C2005F08C10037
:101E000073308316B4008312732566308316B400D2
:101E1000831273258316D22E8312861FAF2F061FBF
:101E2000AF2F8316B201831244088316B7008312C2
:101E300043088316B600831242088316B500831246
:101E400041088316B4008312002078088316B1007D
:101E50003108023C031D362F8312C401C301C201A5
:101E60000130C10073308316B000792F310B792F08
:101E70000310FA018312400CF9003F0CF8003E0CED
:101E8000F70039078316B40083123A088316B500A9
:101E900078080318780FB50783123B088316B6003D
:101EA00079080318790FB60783123C088316B70028
:101EB0007A0803187A0FB70783123C088316BB0011
:101EC00083123B088316BA0083123A088316B900BE
:101ED000831239088316B8003708BF003608BE00E1
:101EE0003508BD003408BC0083122423780883160B
:101EF000B00030086E3C0319812F3008733C031D7D
:101F00008C2F01308312C1070318C20A0319C30AB8
:101F10000319C40AAF2F83163008703C031DB02F7D
:101F20008312C408031D9E2FC308031D9E2FC208E1
:101F3000031D9E2F4108013C0318A72FFF30C10746
:101F4000031CC207031CC307031CC407AF2F62088E
:101F5000C4006108C3006008C2005F08C1008316A6
:061F60008312642E6300F1
:00000001FF
